S01D00006F70656E626C745F73746D3332663330332E656C662E737265639A
S31508000000E8080020AD350008C9350008CD350008D8
S31508000010D1350008D5350008D9350008000000009C
S31508000020000000000000000000000000DD350008A8
S31508000030E135000800000000E53500087B1E0008D1
S31508000040E9350008ED350008F1350008F5350008F2
S31508000050F9350008FD3500080136000805360008A0
S31508000060093600080D36000811360008153600084E
S31508000070193600081D3600082136000825360008FE
S31508000080293600082D3600083136000835360008AE
S31508000090393600083D36000841360008453600085E
S315080000A0493600084D36000851360008553600080E
S315080000B0593600085D3600086136000865360008BE
S315080000C0693600086D36000871360008753600086E
S315080000D0793600087D36000881360008853600081E
S315080000E0893600088D3600089136000895360008CE
S315080000F0993600089D360008A1360008A53600087E
S31508000100000000000000000000000000A9360008FA
S31508000110AD360008B1360008B5360008B93600080D
S31508000120BD360008C1360008C5360008C9360008BD
S31508000130CD360008D1360008000000000000000097
S31508000140D5360008D9360008DD360008000000005C
S315080001500000000000000000000000000000000091
S315080001600000000000000000E1360008E53600083F
S31508000170E93600080000000000000000000000004A
S3150800018000000000ED36000870B504460025002C76
S3150800019001D1012070BD4FF45C70261870780028D4
S315080001A004D128463070204600F0B0FE0320707057
S315080001B00CE01C206843204428300121417005705A
S315080001C00021C170C160016141616D1C6068854292
S315080001D0EFD300250DE01C20684320444FF4E67158
S315080001E00844002141700570C170C1600161416118
S315080001F06D1C60688542EED301202168A1F8400095
S3150800020000202168A1F840002168A1F8440021686F
S31508000210A1F850004FF43F402168A1F840000020A3
S3150800022084F8240001207070002070BD10B5040009
S3150800023001D1012010BD032084F87103204600F087
S315080002400DF8204600F085FE002084F8710310BDE5
S3150800025080B5012100F0CDFF002002BD90F8701393
S31508000260012901D102207047012180F87013026824
S31508000270A2F8401000210268A2F84410032102687F
S31508000280A2F84010002180F8701308467047F8B5A8
S3150800029004460020ADF8000028E048F60F70184024
S315080002A0108004F124052068B0F850102A7911EB63
S315080002B0C20100EB410000F204400088C0F30900C7
S315080002C0E8616969084468610021204600F062FE19
S315080002D0287800280AD0A869002807D1287840F08D
S315080002E080002168A1F84C0000202870216801F1DF
S315080002F044000288ADF80220120440F17281BDF86C
S31508000300022012F00F067AD10A461388BDF8025069
S31508000310ED06C2D5ADF80030BDF800502D051FD545
S315080003204FF4E672A51880892A7810EBC20001EB13
S31508000330400000F20C400088C0F30903AB61AA88AC
S315080003404FF45D702118206800F0B7FF2068018817
S3150800035040F68F7211400180204600F00AFEC5E77C
S31508000360BDF800000004C1D540F68F701840108013
S3150800037020684FF4E6716518B0F850102A7811EB2A
S31508000380C20100EB410000F20C400088C0F30903EB
S31508000390002BAB6108D0AA882969206800F08DFF78
S315080003A02869A969084428610021204600F0E8FD6B
S315080003B02068B0F8501000EB410000F20C40E968E4
S315080003C03F2909D34A0911F01F0F00D1521E910285
S315080003D041F40041018005E04A08C90700D5521CCE
S315080003E091020180206801884BF68F72114081F4D2
S315080003F0405141F4004141F08001018076E701EB6C
S3150800040086000188ADF80010BDF8002012046BD5EF
S3150800041040F68F7211400180C6EBC60004EB8000DF
S315080004204FF4E67145182A78D30020680146AF7A5A
S31508000430002F11D1B0F850209A1801EB420101F2B1
S315080004400C410988C1F30907002F37D03B46AA8813
S31508000450296900F032FF31E030F822205204B0F862
S3150800046050200FD59A1801EB420101F20441098880
S31508000470C1F30907002F14D03B46EA88296900F022
S315080004801CFF0EE09A1801EB420101F20C410988A3
S31508000490C1F30907002F04D03B462A89296900F0D1
S315080004A00CFF2068297800EB8100018848F68F72D6
S315080004B0114041F4004141F0C00101803846A96964
S315080004C04118A9612969CA192A616B69002B02D0EA
S315080004D0E968884204D22978204600F051FD03E0F5
S315080004E02978204600F06AFBBDF8000000067FF573
S315080004F0FDAEC6EBC60004EB800000F128052068B7
S3150800050000EB8600018848F60F72114001802978B1
S31508000510CA0023681846AE7A002E12D1B3F85010D6
S31508000520511800EB410000F204400088C0F30903AB
S31508000530002BAB6139D0AA882969206800F0AAFE89
S3150800054033E013F821104906B3F8501010D55118A6
S3150800055000EB410000F204400088C0F30903002BB9
S31508000560AB6115D0EA882969206800F093FE0FE090
S31508000570511800EB410000F20C400088C0F3090353
S31508000580002BAB6104D02A892969206800F082FE15
S315080005902068297800EB8100018848F68F7211409F
S315080005A041F4404141F0800101802068B0F85010C4
S315080005B02A7811EBC20100EB410000F204400088E2
S315080005C0C0F30900A86129690A182A616B692978A4
S315080005D0002B204602D100F0DDFC87E600F073FB15
S315080005E084E60020F2BD10B504462068B0F8440041
S315080005F0000402D52046FFF74AFE2068B0F84410EA
S3150800060049050AD54FF6FF31A0F84410204600F0F8
S31508000610CEFC0021204600F085F82068B0F844108A
S31508000620490403D54BF6FF71A0F844102068B0F8CA
S315080006304410890403D54DF6FF71A0F844102068CC
S3150800064040308188C90414D501884FF6FB721140E1
S3150800065001802068B0F840104FF6F7721140A0F8F4
S315080006604010204600F0C1FC4EF6FF702168A1F844
S315080006704400206840308188090517D5018841F073
S31508000680080101804FF2FF702168A1F84400206834
S31508000690B0F8401041F00401A0F840102068B0F806
S315080006A04400C00402D4204600F08EFC2068B0F84E
S315080006B04410890506D54FF6FF51A0F84410204688
S315080006C000F071FC2068B0F84410C90503D54FF650
S315080006D0FF61A0F8441010BD10B5044694F87003E5
S315080006E0012801D1022010BD012084F870030146BB
S315080006F0204600F07EFD002084F8700310BD10B57A
S31508000700044694F87003012801D1022010BD012087
S3150800071084F870030021204600F06BFD002084F861
S31508000720700310BD90F87023012A01D1022070478A
S31508000730012280F870230A0004D180210268A2F8F9
S315080007404C1001E080F82410002180F87013084648
S3150800075070470000F0B401F07F04C4EBC40500EB59
S3150800076085040D0601D5283402E04FF4E6752C44BD
S3150800077001F07F052570C9096170E260E37090F8A1
S315080007807013012901D102204CE1012180F8701370
S31508000790E178032930D8DFE801F002240E18217821
S315080007A0026802EB81010A8848F68F131A4042F460
S315080007B000720A8020E02178026802EB81010A882B
S315080007C048F68F131A400A8016E02178026802EB71
S315080007D081010A8848F68F131A4042F4C0620A80DB
S315080007E00AE02178026802EB81010A8848F68F132D
S315080007F01A4042F480620A802378016801EB830577
S3150800080048F2800148F68F722E88164033430B4310
S315080008102B8023780568A67A002E69D1DE00A38886
S315080008204FF6FE773B402F4694F801C0BCF1000F07
S31508000830B5F850501FD0751907EB450505F58065C5
S315080008402B800368257803EB85031D886E0605D57E
S315080008502A4042F4004242F0C0021A800268237815
S3150800086002EB8302138848F6BF74234083F0200303
S3150800087019431180D2E0751907EB450505F5816521
S315080008802B800368B3F85050267815EBC60503EBA2
S31508000890450303F20C43E5683F2D09D36E0915F0AD
S315080008A01F0F00D1761EB50245F400451D8005E0F0
S315080008B06E08ED0700D5761CB5021D8003682578FD
S315080008C003EB85031D886E0405D52A4042F4404291
S315080008D042F080021A800268237802EB83021388AA
S315080008E04BF68F74234083F440531943118095E0E7
S315080008F005EB83031D88154045F4014545F0800541
S315080009001D800368B3F85050267815EBC60503EB2F
S31508000910450303F58063E5884FF6FE7635401D806E
S315080009200368B3F85050267815EBC60503EB450364
S3150800093003F5816325894FF6FE7635401D800368E9
S31508000940257803EB85031D886678002E32D16E0460
S3150800095005D5154045F4404545F080051D800368DA
S31508000960257803EB85052E8848F2C003770602D55D
S3150800097016401E432E800568267805EB86052E88C8
S3150800098032401A432A800268237802EB83021388CE
S315080009904BF68F752B4083F440530B431380026844
S315080009A0237802EB8302138848F6BF742340194361
S315080009B0118033E06E0405D5154045F4404545F0F1
S315080009C080051D800368257803EB85031D886E0660
S315080009D005D5154045F4004545F0C0051D8003685A
S315080009E0257803EB85031D882A4042F4404242F0ED
S315080009F080021A800268237802EB8302138848F67D
S31508000A00BF752B400B4313800268237802EB8302E1
S31508000A1013884BF68F74234019431180002180F800
S31508000A2070130846F0BC704770B401F07F02C2EB41
S31508000A30C20300EB83020B0601D5283202E04FF40D
S31508000A40E6731A4401F07F031370C909517090F8D0
S31508000A507013012901D10220AEE0012180F870133C
S31508000A600168137801EB83010C885578937A002B7B
S31508000A7031D1002D17D0630607D548F68F7323406A
S31508000A8043F4004343F0C0030B800168127801EB7E
S31508000A9082010A8848F6BF731A4042F4004242F0BF
S31508000AA080020A8084E0630407D548F68F732340E2
S31508000AB043F4404343F080030B800168127801EB4E
S31508000AC082010A884BF68F731A4042F4004242F0BC
S31508000AD080020A806CE048F68F73002D32D16504D7
S31508000AE005D51C4044F4404444F080040C80016859
S31508000AF0147801EB84010C8848F2C005660602D515
S31508000B001C402C430C800168147801EB84010C8886
S31508000B1023402B430B800168137801EB830348F2CB
S31508000B2080011C884BF68F752C400C431C8003688B
S31508000B30127803EB8202138848F6BF7423401943E0
S31508000B40118035E0650405D51C4044F4404444F062
S31508000B5080040C800168147801EB84010C88650612
S31508000B6005D51C4044F4004444F0C0040C800168D8
S31508000B70147801EB84010C88234043F4404343F086
S31508000B8080030B800168137801EB830348F2800128
S31508000B901C8848F6BF752C400C431C8003681278E5
S31508000BA003EB820213884BF68F7423401943118096
S31508000BB0002180F87013084670BC704730B401F005
S31508000BC07F04C4EBC40500EB85044FF4E6752C449A
S31508000BD0226163610022A261627001F07F012170C7
S31508000BE06269E168914202D2521A626102E01146D4
S31508000BF000226261A27A002A1CD10268B2F850303B
S31508000C00257813EBC50302EB430202F20C423F2997
S31508000C1009D34B0911F01F0F00D15B1E990241F44D
S31508000C200041118033E04B08C90700D55B1C9902C7
S31508000C3011802CE0627813001CD10268B2F850309B
S31508000C40257813EBC50302EB430202F20C423F2957
S31508000C5009D34B0911F01F0F00D15B1E990241F40D
S31508000C600041118013E04B08C90700D55B1C9902A7
S31508000C7011800CE0012A0AD10268B2F850302578B2
S31508000C8013EBC50302EB430202F20C421180006823
S31508000C90217800EB810001884BF68F72114081F4B0
S31508000CA0405141F4004141F080010180002030BCF0
S31508000CB0704701F07F01C1EBC10200EB8200D0F85A
S31508000CC0E40180B2704770B5044601F07F00C0EBBE
S31508000CD0C00504EB850000F128052A616B61002038
S31508000CE0A8610120687001F07F0028706869EE68C5
S31508000CF0864202D2801B686102E0064600206861CF
S31508000D002068A97A002911D133469BB2AA88296995
S31508000D1000F0C0FA2068B0F850102A7811EBC2012A
S31508000D2000EB410000F2044006802CE0297810F818
S31508000D302110490601D52A8900E0EA8833469BB284
S31508000D40296900F0A7FA687801000DD1287821688A
S31508000D5001EB8000018848F68F72114041F400418A
S31508000D6041F0C00101800EE001280CD128782168E5
S31508000D7001EB8000018848F68F72114041F440412A
S31508000D8041F0800101802068297800EB8100018804
S31508000D9048F6BF72114081F0300141F4004141F03C
S31508000DA080010180002070BD30B490F87023012ABC
S31508000DB001D1022044E0012280F870230A461C2350
S31508000DC00C0607D502F07F0213FB02F2024402F179
S31508000DD0280305E013FB02F202444FF4E6731344BA
S31508000DE001229A7001F07F021A70C90959701C789D
S31508000DF0016801EB84010D8848F28002002C09D1B4
S31508000E004BF6BF732B4083F4805383F010031A43C9
S31508000E100A8011E05B78002B07D048F6BF732B4099
S31508000E2083F010031A430A8006E04BF68F732B40B3
S31508000E3083F480531A430A80002180F87013084609
S31508000E4030BC704710B40A461C230C0606D502F0BF
S31508000E507F0213FB02F20244283205E013FB02F27A
S31508000E6002444FF4E6731A440023937001F07F039B
S31508000E701370C909517090F87013012901D1022025
S31508000E8041E0012180F870130168137801EB8301B2
S31508000E900B885478002C19D05C0607D548F68F7451
S31508000EA0234043F4004343F0C0030B8001681278E3
S31508000EB001EB82010A8848F6BF731A4082F03002B5
S31508000EC042F4004242F080020A8018E05C0407D52A
S31508000ED048F68F74234043F4404343F080030B8065
S31508000EE00168127801EB82010A884BF68F731A4063
S31508000EF082F4405242F4004242F080020A80002105
S31508000F0080F87013084610BC7047000000685E49F8
S31508000F10884200D0704700B587B04FF4C0500190A2
S31508000F200220029000200390032004900E200590D2
S31508000F3001A94FF0904000F0D9F95448016841F4EE
S31508000F4000010160006800F400000090009807B0F6
S31508000F5000BD00684C4988420AD14C48016821F412
S31508000F60000101604FF4C0514FF0904000F06DBA97
S31508000F7070474FF45D710144D0F8A40300F042BBFA
S31508000F80C1EBC10200EB8202D2F8DC21D0F8A4033F
S31508000F9000F065BBC1EBC10200EB8202926BD0F890
S31508000FA0A40300F092BBD0F8A40300F01DBC10B552
S31508000FB004460121D4F8A40300F003FCD4F8A403E2
S31508000FC0BDE8104000F0DABB10B5044600F04CFC52
S31508000FD0D4F8A40300F0F8FBA069002804D02C4834
S31508000FE0016841F00601016010BD80B5D0F8A40380
S31508000FF000F0F3FBBDE8014000F037BC10B504462D
S315080010002448C0F8A443C4F820021F4901600821F7
S315080010104160022181600021C16002210161002135
S3150800102081610162FFF7B0F8002805D040F243114C
S315080010300FF2D01000F01FFC182300221146D4F836
S31508001040200200F009F9582300228021D4F8200252
S3150800105000F002F9C02300228121D4F8200200F012
S31508001060FBF84FF4887300220121D4F8200200F01F
S31508001070F3F84FF4807300228221D4F8200200F09E
S31508001080EBF8002010BD0000005C00401C10024078
S3150800109010ED00E0E808002010B50024D0F8200282
S315080010A0FFF7C4F8002804D0022801D1012400E083
S315080010B00224204610BD10B50024D0F82002FFF700
S315080010C0C7F8002804D0022801D1012400E0022430
S315080010D0204610BD10B50024D0F82002FFF7BEF850
S315080010E0002804D0022801D1012400E00224204669
S315080010F010BD38B51C46002513462246D0F82002F6
S31508001100FFF728FB002804D0022801D1012500E0BA
S315080011100225284632BD10B50024D0F82002FFF774
S3150800112083FC002804D0022801D1012400E002240F
S31508001130204610BD10B50024D0F82002FFF734FE73
S31508001140002804D0022801D1012400E00224204608
S3150800115010BD10B50024D0F82002FFF773FE002852
S3150800116004D0022801D1012400E00224204610BD43
S31508001170D0F8200201F07F02C2EBC20300EB830025
S31508001180090602D590F82A00704790F8CE017047F4
S3150800119010B50024D0F82002FFF7C4FA002804D0BE
S315080011A0022801D1012400E00224204610BD10B512
S315080011B00024D0F82002FFF786FD002804D0022874
S315080011C001D1012400E00224204610BD10B50024F8
S315080011D0D0F82002FFF7F2FC002804D0022801D13B
S315080011E0012400E00224204610BDD0F82002FFF7B3
S315080011F060BD012902D1012000F01ABB002000F0D1
S3150800120017BB0000433A5C576F726B5C4F70656E94
S31508001210424C545C5461726765745C44656D6F5CDE
S3150800122041524D434D345F53544D333246335F4438
S315080012306973636F766572795F4633303356435FF9
S315080012404941525C426F6F745C757362645F636F89
S315080012506E662E630000000030B41C240D0606D509
S3150800126001F07F0114FB01F10844283004E06143D2
S3150800127008444FF4E6710844002A03D1002181721C
S31508001280838004E001218172C380190C018100204A
S3150800129030BC704710B400EB420000F580605A1C61
S315080012A0520807E00B784C7843EA042320F8043BFD
S315080012B0891C521EF6D110BC704710B400EB4200D0
S315080012C000F580605A0806E030F8044B0C70240AD2
S315080012D04C70891C521EF7D103EBD3725210B3EB34
S315080012E0420201D00088087010BC7047F8B400228A
S315080012F025E0052707FA06F646EA0C0645F82460AF
S31508001300914C2668DD432E404F68FF0300D51E43E7
S31508001310266066682E404F68BF0300D51E43666088
S31508001320A6682E404F68FF0200D51E43A660E668F1
S3150800133035404E68B60200D51D43E560521C0B6861
S315080013401C46D44000F07F80012494402340F5D009
S315080013504D68022D01D0122D12D1D50800EB850655
S31508001360356A970007F01C074FF00F0C0CFA07FCBC
S3150800137025EA0C05D1F810C00CFA07F73D4335628B
S31508001380056856000327B740FF433D4091F804C05F
S315080013900CF0030C0CFA06FC4CEA050505604D68D2
S315080013A0012D05D0022D03D0112D01D0122D11D1FA
S315080013B085683D40D1F80CC00CFA06FC4CEA0505D8
S315080013C08560456825EA04044D68C5F3001595400F
S315080013D02C434460C56807EA05048D68B5402C436C
S315080013E0C4604C68E400A9D5584C256845F0010549
S315080013F02560246804F001040094009C9408544D68
S3150800140055F824C0970007F00C060F27B7402CEABA
S31508001410070CB0F1904F01D100276BE74D4FB8424A
S3150800142001D1012766E74C4FB84201D1022761E78F
S315080014304A4FB84201D103275CE7494FB8427FF4C7
S3150800144058AF042756E7F1BC70472DE9F041002252
S315080014501AE04FF0050E0EFA07F7BC4513D154F8FB
S31508001460257027EA060644F82560DB43364C2568CE
S315080014701D40256065681D406560A5681D40A5601E
S31508001480E5682B40E360521C0B46D34054D0012339
S3150800149003FA02F414EA0103F5D003255600B54011
S315080014A0ED4306682E400660D60800EB860C9700CA
S315080014B00F26DCF820E007F01C0806FA08F82EEAE2
S315080014C0080ECCF820E0D0F808C005EA0C0CC0F8E5
S315080014D008C0D0F804C02CEA04044460C4682C4050
S315080014E0C46095081A4C54F825C007F00C07BE408E
S315080014F006EA0C0CB0F1904F02D14FF0000EAAE7A5
S31508001500DFF850E0704502D14FF0010EA3E7DFF88F
S3150800151048E0704502D14FF0020E9CE7DFF83CE048
S31508001520704502D14FF0030E95E7DFF834E07045B9
S315080015308FD14FF0040E8EE7BDE8F081002A01D066
S3150800154081617047816270470004014018100240AB
S31508001550080001400004004800080048000C004844
S315080015600010004810B5002801D1022010BD4FF424
S31508001570FE7303449C69002C01D000249C61002959
S3150800158000D05961012119700270FFF737FD00205C
S3150800159010BD10B504464FF4FE70221801201070D5
S315080015A06168C9B220469269526890472046FFF79B
S315080015B091FD2046FFF770FD002010BD002200298E
S315080015C002D0C0F8141200E002221046704780B517
S315080015D0FFF771FD002002BD0020704710B50224F8
S315080015E0D0F81422002A04D012689047002800D1A7
S315080015F00024204610BD80B5D0F8142252689047C2
S31508001600002002BD38B504464FF402702518284656
S3150800161000F05CFB4FF4FA70204401210160418B15
S315080016204160007D10F01F0103D002290BD005D3BD
S315080016300EE02946204600F023F90EE0294620460A
S3150800164000F042F909E02946204600F059F904E07D
S3150800165000F080012046FFF76DFD002032BD38B549
S31508001660044610464FF4FA7222440B0022D1116840
S31508001670032928D14FF4867121444B680D68AB4283
S315080016800BD2EA1A0A6049688A4200D30A4692B21D
S315080016900146204600F078FB15E0106A016908004B
S315080016A004D0107A032801D120468847204600F046
S315080016B073FB08E0106A8369180004D0107A0328BF
S315080016C001D120469847002032BD38B50446104659
S315080016D04FF4FA72A5180A0045D12968022939D1AA
S315080016E004F118014A688B6893420DD2D21A4A60EF
S315080016F092B20146204600F03FFB00231A461146E7
S315080017002046FFF763FD25E00868B0FBF3F103FB0D
S315080017101101002912D1984210D3696888420DD266
S3150800172000221146204600F027FB00206860034689
S31508001730024601462046FFF749FD0BE0286AC168C4
S31508001740080004D0287A032801D120468847204675
S3150800175000F02DFB287B01280ED12046FFF73CFF21
S315080017600020287308E0286A4269100004D0287A05
S31508001770032801D120469047002032BD10B5044603
S31508001780402300221146FFF7B4FC4020C4F810019C
S315080017900346002280212046FFF7ABFC201D40218E
S315080017A0C1614FF4FE71621801211170D1690029D7
S315080017B005D00168C9B22046926952689047002050
S315080017C010BD0174002070474FF4FE71084401787B
S315080017D0417004210170002070474FF4FE710844DF
S315080017E0417801700020704780B54FF4FE710144BE
S315080017F00A78032A04D18969C9690A0000D088478A
S31508001800002002BD00690840884201D101207047C6
S315080018100020704780B501214FF09040FFF7F2FF96
S31508001820002801D0002002BD00F0F1FA012002BD17
S31508001830012800D1704700B585B04FF4805000905C
S3150800184001200190002002900320039069464FF082
S315080018509040FFF74BFD00224FF480514FF0904027
S31508001860FFF76CFE05B000BD70477047642000F0B6
S31508001870ADBA00F0AEBA80B500F0D4FAFCE70000C5
S3150800188080B54A78092A1BD8DFE802F011171A141E
S315080018901A08051A0E0B00F0C3F813E000F04CF90D
S315080018A010E000F06EF90DE000F0B6F90AE000F07D
S315080018B0C9F907E000F0DAF904E000F0EBF901E015
S315080018C000F018FA002002BD38B504460D464FF45C
S315080018D0FE702218107803280DD1287902280ADA12
S315080018E02046926992689047E888002806D12046E3
S315080018F000F052FA02E0204600F0FCF9002032BD62
S3150800190070B504460D462979287800F0600020282D
S3150800191009D1294620464FF4FE72224492699268FC
S315080019209047002070BD687800284AD0012825D045
S31508001930032873D14FF4FE7026183078022802D097
S31508001940032808D066E0002968D0802966D020469A
S31508001950FFF7F0FB62E06888002806D1002904D06A
S31508001960802902D02046FFF7E5FB29462046B269C2
S3150800197092689047204600F00FFA4FE04FF4FE7049
S3150800198026183078022802D0032808D042E0002919
S3150800199044D0802942D02046FFF7CCFB3EE0688839
S315080019A000283BD111F07F0007D02046FFF7D1FB76
S315080019B029462046B26992689047204600F0ECF91D
S315080019C02CE094F8FC01022802D0032807D021E075
S315080019D011F07F0022D02046FFF7ACFB1EE001F095
S315080019E07F0004EB00100A46120602D500F1140522
S315080019F002E04FF4827285182046FFF7B9FB401EB5
S31508001A008041C043C00F286002222946204600F0C4
S31508001A10A4F903E02946204600F06CF9002070BDC1
S31508001A2038B504460D4669880846000A401E062849
S31508001A3000F27D80DFE800F0041F317B7B636E00D7
S31508001A406946207CD4F8102212689047BDF8001029
S31508001A5000290FD0E9880A000CD0BDF800208A4278
S31508001A6000D90A46ADF80020BDF8002001462046F8
S31508001A7000F073F931BD4FF4047020444168207CAE
S31508001A800028684604D1896A884702214170DDE743
S31508001A90C96A884702214170D8E7C9B2052946D8DC
S31508001AA0DFE801F0030A11181F266946207CD4F8DE
S31508001AB0102252689047C9E76946207CD4F810225C
S31508001AC092689047C2E76946207CD4F81022D2680B
S31508001AD09047BBE76946207CD4F8102212699047E4
S31508001AE0B4E76946207CD4F8102252699047ADE7DE
S31508001AF06946207CD4F8102292699047A6E7207C94
S31508001B00002814D168464FF4047121444968496B8A
S31508001B1088479BE7207C002809D168464FF4047162
S31508001B2021444968096B8847072141708EE7294691
S31508001B30204600F0DFF831BD70B5044688880028D5
S31508001B401BD1C888002818D1887800F07F054FF483
S31508001B50FE702618307803280FD0B570294620461F
S31508001B60FFF716FB204600F017F9002D02D00220D9
S31508001B70307070BD0120307070BD2046BDE87040E1
S31508001B80B8E070B504460D46224E68883070317844
S31508001B9002293ADA94F8FC01022802D0032810D068
S31508001BA033E0080008D06160032084F8FC01204671
S31508001BB0FFF714FD022823D02046BDE8704000F048
S31508001BC0EBB808000DD1022084F8FC010020606003
S31508001BD001462046FFF70FFD2046BDE8704000F09D
S31508001BE0DBB860688142E7D00146C9B22046FFF7F4
S31508001BF002FD317861602046FFF7F0FC0228DBD150
S31508001C0029462046BDE8704074E029462046BDE8CE
S31508001C1070406FE0BC160020CA88012A11D190F8DE
S31508001C20FC21022A02D0032A07D00AE0002181609B
S31508001C30012200F1080100F090B80122011D00F010
S31508001C408CB857E04FF4FE72024413789B1E012BA2
S31508001C500BD80121C1609168002901D00321C16018
S31508001C60022200F10C0100F078B843E010B50446F2
S31508001C70488801280DD14FF4017022180120106000
S31508001C8020461269926890472046BDE8104000F049
S31508001C9083B810BD10B504464FF4FE7022181078AC
S31508001CA0801E01280DD8488801280ED10020906092
S31508001CB020469269926890472046BDE8104000F099
S31508001CC06BB82046BDE8104014E010BD0A780270D3
S31508001CD04A7842708A78CB7812EB032242800A79D6
S31508001CE04B7912EB032282808A79C97912EB01219A
S31508001CF0C180704710B504468021FFF71BFA002102
S31508001D002046BDE81040FFF715BA70B504460D46E3
S31508001D101646002C16D000F016F84000801C3080BD
S31508001D203088287003206870022008E014F8011B28
S31508001D30C0B22954401C0021C0B22954401C217845
S31508001D400029F3D170BD002101E0491C401C02782E
S31508001D50002AFAD10846C0B2704780B50223C0F8F7
S31508001D60F43100F118031A605A6013460A46002136
S31508001D70FFF71DFA002002BD80B513460A4600216A
S31508001D80FFF715FA002002BD80B513460A46002162
S31508001D90FFF71CFA002002BD80B50421C0F8F41133
S31508001DA000231A461146FFF702FA002002BD80B545
S31508001DB00521C0F8F41100231A461146FFF706FA62
S31508001DC0002002BD816170478162704712494880D0
S31508001DD0704710B500F043F80F4C6168884215D378
S31508001DE00E482178002906D1012121704FF480710F
S31508001DF0FFF7E8FF05E0002121704FF48071FFF737
S31508001E00E3FF00F02CF861884018606010BD4FF4BD
S31508001E1080710248D8E70000B0160020001000487C
S31508001E20FFF724BDFFF725BD80B500F00BF80F4876
S31508001E300F494160002181600521016000200D499C
S31508001E40086001BD00200949086070470748006816
S31508001E50C00303D507480168491C0160704780B56F
S31508001E60FFF7F4FF0348006802BD000010E000E039
S31508001E703F190100B8160020F1E77047DFF88C0318
S31508001E800021018000F1440100224A6080F84320C5
S31508001E900A80114681707047DFF870030178481E82
S31508001EA08041C043C00F70470020DFF8601381F8F7
S31508001EB04300704710B50178D44CFF2914D100F0BF
S31508001EC084F894F84300012802D1102000F074F831
S31508001ED0B4F94410012906DB012084F84300E01C0C
S31508001EE0BDE810404EE010BD2278012AFBD1C92971
S31508001EF032D0CC293FD0CF293AD0D0292FD0D129DA
S31508001F0033D0D2292ED0F32917D0F4290FD0F529AA
S31508001F100AD0F6290ED0FA2912D0FC2913D0FD29A9
S31508001F2014D0FE2915D029E000F0A7F8C9E700F07B
S31508001F30C1F8C6E700F098F8C3E700F0DAF8C0E79A
S31508001F4000F081F8BDE700F07CF8BAE700F069F820
S31508001F50B7E700F05AF8B4E700F0F1F8B1E700F097
S31508001F600BF9AEE700F0D8F8ABE700F032F9A8E7CE
S31508001F7000F042F9A5E700F04BF9A2E7202000F0AF
S31508001F801BF89EE789B200F065B9F8B504460D4618
S31508001F901646002705E02078C719FFB2641CFFF72C
S31508001FA041FF2846451E0028F5D137600120F2BDBD
S31508001FB000209649487070479449CA1CFE2313703E
S31508001FC050700220A1F84400704710B5FFF7F0FFE3
S31508001FD08E4C01202070FF20E07010202071002018
S31508001FE0607100F045F9A07100F050F9E07100F059
S31508001FF04DF9000A207201206072A0720820A4F828
S315080020004400BDE8104000F053B910B57F4C0020DD
S315080020102070FFF7CDFFFF20E0700120A4F84400F0
S3150800202010BD7A48411CFF228A700022CA700A78BD
S315080020300A7100224A718A71CA710621A0F84410F1
S3150800204070470020B8E77148C11CFF220A70443067
S315080020500FF2C012426000224A708A70CA700722C4
S315080020604A600821018070476849FF22CA704431D6
S315080020704068486001200880704770B5054600F042
S31508002080F7F86A78401E904203DA2220BDE87040CD
S3150800209092E75E4E06F144046168301D00F042F98D
S315080020A0FF20F07060686978401860606878401CA6
S315080020B0208070BD70B5044600F0DAF8401E6178DD
S315080020C0884203DA2220BDE8704075E761684F4E02
S315080020D006F1440569606278301D00F023F9FF2097
S315080020E0F07068686178401868606078401C2880DD
S315080020F070BD38B54549CC1CFF22227001F1440554
S31508002100CA1D41686868FFF740FF60700020A0702C
S31508002110E0700820288031BD38B53C4CE51CFF200E
S31508002120287000206870A87000F0A2F8E8700020F7
S3150800213028716871A8710720A4F8440031BD70B5EC
S31508002140054600F095F8314E06F144046A1C411E16
S31508002150606800F0AFF8002803D13120BDE8704070
S315080021602AE7FF20F07000F083F86168401E4018E7
S3150800217060600120208070BD38B5044600F078F80C
S31508002180801E6178884203DA2220BDE8324013E7D0
S315080021901E48FF21C17000F144050120288061789E
S315080021A0080007D100F08EF8002811D13120BDE8CB
S315080021B0324001E7A21C686800F07CF8002803D1C9
S315080021C03120BDE83240F7E66868617840186860F3
S315080021D031BD38B50D4C04F144054168686800F016
S315080021E06BF8002803D13120BDE83240E4E6FF2031
S315080021F0E0700120288031BD80B500F071F80348F1
S31508002200FF21C1700121A0F8441001BDBC140020B3
S315080022103120D1E64F70656E424C540080B5FFF709
S315080022202DFE00F091F802201F49087001BD10B577
S3150800223082B01D4C6946201D00F0E7F8012806D13A
S31508002240022020709DF80010201DFFF733FE13BDF5
S3150800225000F0A6B8144A1278022A01D0FFF724BE65
S3150800226080B5C9B200F0A7F8BDE80140FFF71CBE6B
S315080022700D480078012805D006D3032802D003D2DA
S315080022803F20704700207047402070470648007876
S31508002290012805D006D3032802D003D23F20704771
S315080022A0002070474020704700000020FFF7F4BD6B
S315080022B000F0EEB900F0F3B900F00FBA00F066BA14
S315080022C000F090BA80B500F043FA002801D100204A
S315080022D002BDBDE8014000F06EBA000000F023BB65
S315080022E010B5FFF7EBFF002816D0FFF793FA002882
S315080022F012D0FFF7ADFFFFF7A5FD00F029FBFFF7AA
S31508002300DFFF0649084006490860FFF7D9FF001DA8
S31508002310046800F00AFBA04710BD000080FFFF1FFD
S3150800232008ED00E070B504460D46164605E015F8BA
S31508002330010B04F8010BFFF775FD3046461E80B207
S315080023400028F4D170BD000038B500F0EFF8BB4C9A
S315080023504021601C00F0FFF82070B94D4021681C30
S3150800236000F0F9F828702178FF2901D0FF2804D158
S3150800237073210FF2E820FFF77EFAB24C0022B24929
S315080023802046FFF7EFF8B1492046FFF717F9204630
S31508002390FFF71DF9D4F82002BDE83240FEF79CB9D4
S315080023A010B5A84CD4F82002FEF7A9F92046BDE8D6
S315080023B01040FFF7EEB870B504460D46402D04DB15
S315080023C09B210FF29820FFF756FA284600F057F897
S315080023D0012804D09F210FF28420FFF74CFA00262B
S315080023E00DE0FFF71FFDB6B2A05D00F048F8012822
S315080023F004D0A8210FF26420FFF73DFA761C304678
S31508002400294680B28842ECD370BD70B505460E46A3
S315080024108C48D0F82002FEF7E6F88D4C6078002844
S315080024200FD1201D00F027F8012808D120790100D6
S3150800243005D0402803DA01206070002020700020B3
S3150800244070BD20782044401D00F015F80128F6D10B
S315080024502078421C227010462179C0B28842EED1FB
S31508002460D2B2611D2846FFF75DFF00206070207814
S315080024703070012070BD014671480078A6E001461B
S315080024806E4800787CE0F8B56C4C207800F0C4F80B
S3150800249005001FD0412D00DB4025002610E06946C7
S315080024A0207800F093F8012805D04FF494710FF2C4
S315080024B0AC10FFF7E0F99DF800006649C855761C90
S315080024C0F6B23746AF42EADB2B46624A81215D48BF
S315080024D0FEF76DFEF1BDF8B5044600F0BAFA0546FA
S315080024E0584E21463046FEF780FE0446A4B2002721
S315080024F00DE0295C5248007800F042F8012805D022
S315080025004FF4A5710FF25410FFF7B5F97F1CBFB24F
S315080025103846A042EDDB00F09CFA40230246012132
S31508002520304601B0BDE8F040FEF750BE10B44A4848
S31508002530014600F11802002305E000238B744A6166
S315080025401831183201231C00F7D08B7400224A6117
S31508002550006310BC704710B43F4A136B002B01D1BF
S31508002560FF200BE05C69146319749860D860002238
S315080025705A7418600844401E5860987C10BC70470E
S3150800258038B505460C46022D05DB4FF4D1710FF21E
S31508002590CC00FFF770F9304805EB450100EBC100A8
S315080025A0417C027C914201D1002032BDC1680C7089
S315080025B0417C491C4174C168491CC1604168C268B4
S315080025C0914201D20168C160012032BD38B5054685
S315080025D00C46022D05DB4FF4E2710FF28000FFF77F
S315080025E04AF91D4805EB450100EBC100417C00296D
S315080025F001D1002032BD816809782170417C491ECD
S3150800260041748168491C816041688268914201D29F
S3150800261001688160012032BD10B50446022C05DB35
S315080026204FF4F2710FF23400FFF725F90A4804EB6C
S31508002630440100EBC100407C10BD000008150020D5
S315080026404C150020900C0020B000002078000020D7
S3150800265090150020D415002054160020433A5C57E4
S315080026606F726B5C4F70656E424C545C5461726756
S3150800267065745C536F757263655C41524D434D34A6
S315080026805F53544D333246335C7573622E630000D4
S315080026904FF0FF306C4908606C490860704730B4E9
S315080026A06B4B1B1A4C1EA34207D36A4B984204D3A2
S315080026B00C18641E684DAC4201D300200BE0440A96
S315080026C064029C420B46014602D1604830BCC7E012
S315080026D05D4830BCC4E030BC70477FB50022039229
S315080026E001245B4A121A4B1E9A4209D3C20AD20225
S315080026F0584B9A4204D30818411E574B994201D3A6
S31508002700002023E0801AC50AADB2400501D06D1C31
S31508002710ADB20020009001922046029000F0EAF93E
S31508002720002604E0019800F500600190761CB6B218
S31508002730AE4208DAFFF776FB03A9684600F042FACC
S315080027400028EFD0002400F0E1F9204604B070BD5F
S3150800275080B53E48016811F1010F01D1012002BD83
S31508002760416882685118C26851180269511842694D
S31508002770511882695118C0694018C043401C00901E
S315080027806A4604213548FFF78AFF02BD31480168C9
S315080027904268511882685118C2685118026951185E
S315080027A042695118806940182C4909680818401E62
S315080027B08041C00F704780B52448016811F1010FA8
S315080027C003D000F08BF8002808D01F48016811F1E3
S315080027D0010F05D000F082F8002801D1002002BDC3
S315080027E0012002BD1B48704780B5CA0501D00020EC
S315080027F002BD02688A4201D1012002BD01604FF480
S315080028000072001DFFF78EFD012002BD38B5044693
S315080028100D460E48844208D10B4C29462046FFF740
S31508002820E3FF00280DD1002032BD0A498D4201D1AF
S315080028300446F2E7204600F051F80028EDD10020C2
S3150800284032BD204632BD0000B40E0020B81000206C
S31508002850FFFF03080040000800000408884100083C
S315080028602DE9F0410746884614461D464FEA582684
S315080028707602386810F1010F05D131463846FFF760
S31508002880B3FF00281DD03868B04205D03146384617
S31508002890FFF7BCFF070014D03868A8EB00003844DF
S315080028A000F10408FFF7BEFA381DA8EB0000B0F5E2
S315080028B0007F0AD306F500713846FFF7A7FF070021
S315080028C001D1002008E007F1040814F8010B08F804
S315080028D0010B6D1EE6D10120BDE8F0812DE9F0411E
S315080028E00546012600F006F9002700E07F1C802F28
S315080028F014D2296801EB870805EB87004468FFF7BF
S3150800290091FA224600234146022000F0ADF800283D
S3150800291003D1D8F80000A042E8D0002600F0F6F867
S315080029203046BDE8F08172B6704762B6704700005F
S3150800293080B50F48016841F010010160032000F0DE
S31508002940FBF9002000F014FA00F0F6FA002002BDA8
S3150800295080B508484FF0FF314160002242600160AF
S315080029600260C1611146C16100F017FB002002BD7B
S31508002970002002400C10024010B5044640230222F3
S315080029808121FEF7B6FB4023022201212046FEF7ED
S31508002990B0FB4023304A01212046FEF717FC0020F1
S315080029A010BD10B504468121FEF7B5FB012120466E
S315080029B0FEF7B1FB002010BD70B50B46172227495C
S315080029C001F10D041D786026354224D15D78062D67
S315080029D004D00A2D10D00B2D12D01CE05D882D0ACC
S315080029E0212D05D101F11604D988182900DA0A46DD
S315080029F02146FFF7B2F90EE00122FFF7AEF90AE029
S31508002A005A881446E4B2002C02D1D2B20A6002E017
S31508002A101946FFF76FF9002070BD80B5FFF733FD43
S31508002A20002002BD80B50846FFF755FD002002BD0F
S31508002A3080B590F8FC01032801D1FFF724FD00209A
S31508002A4002BD20210180064870470A2101800548F9
S31508002A5070470148704700001416002054000020F3
S31508002A6058000020480000202DE9F04780468A4695
S31508002A7014461D464D4E307E012801D1022037E00E
S31508002A80012030764CF25037384600F050F80100F5
S31508002A902CD1B8F1010F02D14FF0010807E0B8F1C7
S31508002AA0020F02D14FF0020801E04FF004084FF080
S31508002AB0000903E009F101095FFA89F9C14515DA48
S31508002AC0204629464FEA091200F0BAFA014689B2A9
S31508002AD00AEB490000F021F8384600F028F8344996
S31508002AE00A68520852000A600100E3D000213176D4
S31508002AF0BDE8F0873048C168090605D52F49016049
S31508002B002F49016000207047012070472848016856
S31508002B1041F080010160002070470022234BDA61F2
S31508002B20234A136843F0010313600180704738B5E0
S31508002B300446FFF7A1F905461E480168C9070BD5E3
S31508002B4014F1010FF8D0002C04D0FFF795F9401BBB
S31508002B508442F1D2032032BD0168890601D52021BD
S31508002B6001600168C90602D40068400703D500F071
S31508002B7004F8012032BD002032BD00200D490A6844
S31508002B80D20605D5094AD06940F00200D061102066
S31508002B900A68520706D5054AD36943F00103D3618B
S31508002BA040F0040008607047000000008816002006
S31508002BB0102002400C2002400420024023016745F1
S31508002BC0AB89EFCD2DE9F84304460D460126DFF81B
S31508002BD0C470387E012801D102203EE0304638769E
S31508002BE04CF2503820680128404610D1FFF79FFF65
S31508002BF000282FD100F033F84046FFF798FF064625
S31508002C00DFF89400016821F00401016022E0FFF773
S31508002C108EFF00281ED14FF0FF302860D4F80490AC
S31508002C2001E009F50069A068616801EBC0208145EB
S31508002C3010D2484600F020F84046FFF778FF0646CF
S31508002C40DFF85400016821F0020101603000E8D085
S31508002C50C5F80090002038763046BDE8F28300209B
S31508002C600C49C8610C48016841F00401016001681B
S31508002C7041F04001016070470021064AD1610649CA
S31508002C800A6842F002020A604860086840F040009C
S31508002C900860704788160020102002402F490A68ED
S31508002CA04FF6FF031A40000200F4E06010432C4A76
S31508002CB010430860704729480068C0F3022070472F
S31508002CC00901002806D5274A00F00F00104400F82D
S31508002CD0041C7047244A1154704710B400F00700CA
S31508002CE0C0F10703052B00D30423041D072C01D2CA
S31508002CF0002000E0C01E012404FA03F35B1E1940FD
S31508002D00814004FA00F0401E1040084310BC70478A
S31508002D1010B5401EB0F1807F01D3012010BD134CC1
S31508002D2060600F214FF0FF30FFF7CAFF0020A06058
S31508002D3007202060002010BDB0E770B504460D4698
S31508002D401646FFF7B8FF32462946FFF7C6FF014683
S31508002D502046BDE87040B3E7DAE700000CED00E076
S31508002D600000FA0518ED00E000E400E010E000E0DD
S31508002D7010B50446074800684FF47A71B0FBF1F0C5
S31508002D80FFF7EAFF002221464FF0FF30FFF7D5FF95
S31508002D90002010BD440000208F48016841F48021BE
S31508002DA0016070478C48016841F4803101607047C2
S31508002DB089480068400C00F00100704787490A6896
S31508002DC0920850EA8200086070478448006800F05C
S31508002DD00C00704781490A6822F0F0021043086027
S31508002DE070477E490A6822F4E0621043086070471B
S31508002DF07A490A6822F46052104308607047774996
S31508002E000A6822F480021043086070477248016815
S31508002E1041F08071016070476F480068400E00F00D
S31508002E200100704710B46D4A136823F4741300F454
S31508002E308034234319431160916A090900F00F0091
S31508002E4050EA0110906210BC704781B064490A6864
S31508002E5002430A60096808400090009801B070476C
S31508002E605F490A6822EA00000860704781B05D4938
S31508002E700A6802430A60096808400090009801B091
S31508002E80704758490A6822EA0000086070475649A0
S31508002E900A68D20850EAC2000860704752480068BB
S31508002EA000F0070070478162704780B500F005F8AA
S31508002EB000F0D5F800F0E2F8FCE780B5FFF738FD3A
S31508002EC0BDE8014080B50220FFF7E1FFFFF7E6FF06
S31508002ED0022804D067210FF21C10FEF7CCFCFFF77E
S31508002EE05BFFFFF75FFFFFF763FF0128FBD14FF496
S31508002EF0E0114FF48030FFF795FFFFF787FFFFF7E4
S31508002F008BFF0128FBD10020FFF764FF4FF4806098
S31508002F10FFF767FF0020FFF76BFF0220FFF74EFF62
S31508002F20FFF753FF0828FBD10020FFF768FF2F485B
S31508002F30BDE8024000F0AEB810B586B00120FFF734
S31508002F4095FF4FF48000FFF780FF4FF40030FFF73E
S31508002F507CFF4FF40010FFF778FF4FF48070009065
S31508002F60012001900020029003900490204C6946AD
S31508002F70204600F069F94FF480712046FFF793FF69
S31508002F8001200090002001900220049069464FF02D
S31508002F90904000F059F906B010BD10B5144C4FF426
S31508002FA080712046FFF77FFF204600F0F4F84FF0C7
S31508002FB0904000F0F0F84FF40010FFF751FF4FF47F
S31508002FC00030FFF74DFF4FF48000FFF749FF01205F
S31508002FD0BDE8104055E7000000100240041002400A
S31508002FE014100240181002400020024000A24A04B1
S31508002FF000100048433A5C576F726B5C4F70656E01
S31508003000424C545C5461726765745C44656D6F5CD0
S3150800301041524D434D345F53544D333246335F442A
S315080030206973636F766572795F4633303356435FEB
S315080030304941525C426F6F745C6D61696E2E630024
S31508003040D2B2203A22BF21FA02F00021704720327C
S31508003050D141D04048409140D1404840704780B562
S31508003060FFF73CF9FEF7DCFEFEF7DEFEFFF720F978
S31508003070FFF7D4F8BDE8014000F02AB980B5FEF79D
S31508003080D1FEFEF7E3FEFFF7D2F8BDE8014000F0F7
S3150800309028B9000001490860704700004400002074
S315080030A030B40368032491FAA1F5B5FA85F56D00E5
S315080030B0AC40A34391FAA1F1B1FA81F1490002FAB1
S315080030C001F11943016030BC704743688B43514393
S315080030D019434160704730B48368032491FAA1F517
S315080030E0B5FA85F56D00AC40A34391FAA1F1B1FAA2
S315080030F081F1490002FA01F11943816030BC704739
S3150800310030B4C368032491FAA1F5B5FA85F56D00C4
S31508003110AC40A34391FAA1F1B1FA81F1490002FA50
S3150800312001F11943C16030BC704730B4036A0F24FB
S3150800313091FAA1F5B5FA85F5AD00AC40A34391FA2D
S31508003140A1F1B1FA81F1890002FA01F1194301628C
S3150800315030BC704730B4436A090A0F2491FAA1F5C6
S31508003160B5FA85F5AD00AC40A34391FAA1F1B1FAE1
S3150800317081F1890002FA01F11943416230BC7047B6
S315080031802B490A6810430860704729490A6822EAE9
S3150800319000000860704710B50124B0F1904F08D1BF
S315080031A04FF40030FFF7ECFF4FF40030FFF7EDFF68
S315080031B03CE02049884208D14FF48020FFF7E0FF21
S315080031C04FF48020FFF7E1FF30E01B49884208D121
S315080031D04FF40020FFF7D4FF4FF40020FFF7D5FF88
S315080031E024E01649884208D14FF48010FFF7C8FF3B
S315080031F04FF48010FFF7C9FF18E01149884208D13B
S315080032004FF40010FFF7BCFF4FF40010FFF7BDFFA7
S315080032100CE00C49884208D14FF48000FFF7B0FF54
S315080032204FF48000FFF7B1FF00E00024204610BDF0
S31508003230281002400004004800080048000C004816
S315080032400010004800140048F8B504460D462868E2
S3150800325090FAA0F0B0FA80F602E0FFF77BFF761C42
S3150800326029680846F04027D00120B04010EA010737
S31508003270F5D06A6839462046FFF712FF68680128C4
S3150800328001D0022804D1AA6839462046FFF723FF51
S315080032902A6939462046FFF733FF68680228DED1D7
S315080032A097FAA7F0B0FA80F008286A6939462046E6
S315080032B0D3D2FFF73AFFD2E76868012801D002287F
S315080032C003D1EA682046FFF700FF0120F2BD00009F
S315080032D010B50F4C01202070FEF7C1FD6060BDE8F7
S315080032E0104010B5FEF7E2FF012810D0084C2078F0
S315080032F001280CD1FEF7B3FD616801F5FA61884231
S3150800330005D300202070BDE81040FEF7E9BF10BDC8
S31508003310A816002012200880274870470420088035
S315080033202648704710B50FF29C03254C00280A461C
S315080033302146184602D1FEF7E8FC01E0FEF7E5FC57
S31508003340204610BD10B51E4C0A4621460FF28800CD
S31508003350FEF7DBFC204610BD10B50FF28C03184CA7
S3150800336000280A462146184602D1FEF7CEFC01E09F
S31508003370FEF7CBFC204610BD10B50FF27C03104CAF
S3150800338000280A462146184602D1FEF7BEFC01E08F
S31508003390FEF7BBFC204610BD10B50FF26403084CBF
S315080033A000280A462146184602D1FEF7AEFC01E07F
S315080033B0FEF7ABFC204610BDCC000020E000002044
S315080033C0BC12002057696E5553422042756C6B201B
S315080033D044657669636500004F70656E424C5420FB
S315080033E055736572000000003030303030303030B0
S315080033F0303530430000000044656661756C740022
S3150800340057696E5553422042756C6B20496E746538
S3150800341072666163650000001448016841F4700132
S3150800342001601348016841F0010101604168114AD1
S31508003430114041600168104A11400160016821F499
S3150800344080210160416821F4FE014160C16A0909D1
S315080034500901C162016B094A1140016300218160BB
S315080034604FF00060064908607047000088ED00E0EC
S31508003470001002400CC07FF8FFFFF6FECCFC00FFF0
S3150800348008ED00E019E050F8041BCB0744BFA9F18A
S3150800349001035918121F0023042A41F8043BF9D2E4
S315080034A05FEA827C0B4604D54FF0000CA1F800C0F9
S315080034B09B1CD10744BF0021197050F8042B002A21
S315080034C0E1D1704730B5016842688468014401EB70
S315080034D05203D20748BF4C44994201D10C3030BD43
S315080034E011F9012B11F8015B002A04F8015B02D5DA
S315080034F0521CF9D1F0E7521EF4D5EDE710B507498D
S3150800350079441831064C7C44163404E00A68081DD0
S31508003510114488470146A142F8D110BD2C0000008D
S31508003520480000004EF68851CEF20001086840F4C3
S3150800353070000860BFF34F8FBFF36F8F4FF00070B6
S31508003540E1EE100A704700003DFFFFFFD80D0000AE
S31508003550E8080020000000006DFFFFFF940100004E
S31508003560220100000000002000F00BF8002801D01E
S31508003570FFF7C4FF0020AFF30080FFF796FC00F0CA
S3150800358002F80120704700F001B8000007463846E7
S3150800359000F002F8FBE7000080B5AFF30080024AAE
S315080035A011001820ABBEFBE7260002000148804741
S315080035B00148004719340008BD350008AFF30080FC
S315080035C0FFF7B0FFFFF7D0FFFFF7FEBFFFF7FEBF1D
S315080035D0FFF7FEBFFFF7FEBFFFF7FEBFFFF7FEBF11
S315080035E0FFF7FEBFFFF7FEBFFFF7FEBFFFF7FEBF01
S315080035F0FFF7FEBFFFF7FEBFFFF7FEBFFFF7FEBFF1
S31508003600FFF7FEBFFFF7FEBFFFF7FEBFFFF7FEBFE0
S31508003610FFF7FEBFFFF7FEBFFFF7FEBFFFF7FEBFD0
S31508003620FFF7FEBFFFF7FEBFFFF7FEBFFFF7FEBFC0
S31508003630FFF7FEBFFFF7FEBFFFF7FEBFFFF7FEBFB0
S31508003640FFF7FEBFFFF7FEBFFFF7FEBFFFF7FEBFA0
S31508003650FFF7FEBFFFF7FEBFFFF7FEBFFFF7FEBF90
S31508003660FFF7FEBFFFF7FEBFFFF7FEBFFFF7FEBF80
S31508003670FFF7FEBFFFF7FEBFFFF7FEBFFFF7FEBF70
S31508003680FFF7FEBFFFF7FEBFFFF7FEBFFFF7FEBF60
S31508003690FFF7FEBFFFF7FEBFFFF7FEBFFFF7FEBF50
S315080036A0FFF7FEBFFFF7FEBFFFF7FEBFFFF7FEBF40
S315080036B0FFF7FEBFFFF7FEBFFFF7FEBFFFF7FEBF30
S315080036C0FFF7FEBFFFF7FEBFFFF7FEBFFFF7FEBF20
S315080036D0FFF7FEBFFFF7FEBFFFF7FEBFFFF7FEBF10
S315080036E0FFF7FEBFFFF7FEBFFFF7FEBFFFF7FEBF00
S315080036F00004BC0006127A000A061001FD0001400B
S3150800370001F9000E09022000010100C03209040077
S315080037100002FFFD0019070581024000FF070501A9
S31508003720024000FF79290008A3290008B9290008E2
S31508003730F8000B1B2A0008252A0008312A0008F47D
S315080037400003432A0008FC00234B2A00081533000F
S31508003750081D33000845330008253300085933008F
S3150800376008793300089933000812011001FD00108A
S3150800377040501DAC6000010102030100000403096A
S306080037800436
S705080035BD00
